:1000000000308A00FC2800000A108A100A118207BA
:1000100028340C34013406340A108A100A1182077D
:10002000413468346F346A342C34203444346934B5
:10003000733470346C3461347934203466347534FC
:100040006E34673475346A34653400342330840088
:10005000000803193A280130F800F701F70B2E28A1
:10006000F80B2D284A30F700F70B34280000000069
:10007000800B2B28003429183F288611402886152C
:10008000831686118312A9184728061148280615D9
:1000900083160611831229194F28861050288614BA
:1000A000831686108312A91957280610582806149B
:1000B0008316061083128617831686130000831298
:1000C00086138316861383120034A708031D6A283B
:1000D00087136B288717A0132008831687008312C5
:1000E000A80E2808A9003B20A80E2808A9003B203C
:1000F0000D30F700F70B7A2800341430A3002620C7
:100100008713A01320088316870083128613831693
:1001100086138312A1012108023C031C9728023098
:10012000A30026200330A9003B20A10A8B280D3014
:10013000F700F70B99280230A9003B200D30F7009B
:10014000F70BA028A1012108023C031CB3282108B9
:100150000420A200A7012208A80065200230A30005
:100160002620A10AA3288A110A123329013023026A
:10017000A5002408023C031DBF284030A507250820
:100180008038A600A7012608A800652000342208B0
:100190000C3A0319D528063A0319DD28073A031942
:1001A000E328053A0319E828ED28A7010130A80043
:1001B00065200230A3002620F9280130A300023078
:1001C000A400B620F9280130A300A400B620F92825
:1001D000A7011030A8006520F92822081F3C031C45
:1001E000F3280730A2050130A7002208A8006520E7
:1001F000F9288A110A12442984011F3083058316C5
:100200001F149F141F159F11FF308312A000831627
:100210001F149F141F159F1183121F10831609129C
:1002200083129412A01220088316870083122016CE
:100230002008831687008312A011200883168700E8
:10024000003083129400831694000108C7390838DF
:100250008100831290010030F80092000030831674
:10026000920083127D2833296430A30026200130B8
:10027000A300A400B620A10121080C200038031916
:0C0280004529A10AA200C7283C29630000
:02400E00393F38
:00000001FF
